:1000000000308A00B6280000831A0A28A500030ED3
:10001000A6000F288312A500030EA600A6140A0846
:10002000AD008A018313A50E0408A7002008A800CC
:100030002108A9002208AA002308AB002408AC006C
:1000400083128B1E25280B194F28270884002808A7
:10005000A0002908A1002A08A2002B08A3002C0850
:10006000A4002D088A00260E83008312250EA618F0
:10007000831609003D08A1013C02031842283C08F0
:10008000A0004E28A0010830BE00BC0DA00D3D0808
:1000900020020318A000A10DBE0B45285F280630E2
:1000A0008100320831020318582830088500592889
:1000B0008501B10A3108BC000930BD003A2820088A
:1000C000B1000B118A11252835308400000803196E
:1000D00076280230A100A001A00B6C28A10B6B2890
:1000E0009730A000A00B7228800B692800343708D5
:1000F00039068039BB00B71F8228B609B709B60A8E
:100100000319B70AB91F8928B809B909B80A031928
:10011000B90AA101A201A001A3013908031D932876
:1001200038080319AD281030BA000310B60DB70D0A
:10013000A00DA30D39082302031DA02838082002B2
:10014000031CA9283808A002031CA3033908A30232
:100150000314A10DA20DBA0B95280000BB1FB528F2
:10016000A109A209A10A0319A20A003484011F30BF
:1001700083051F1383161F149F141F159F15073027
:1001800083129F00703083168F000730831299000E
:100190008316050806308312A000A00BCD280000AE
:1001A00019088C11703083168F0083121F13831669
:1001B0001F109F101F119F110108C03902388100C4
:1001C0000830650083128B16C0308B040630810026
:1001D000B2013208B100B3013308023C031CFE280F
:1001E00005150230B400FA30B5006420B40BF328D2
:1001F0000511C830B5006420B30AEC28851DFE281F
:100200008B12AF01AE01851D10290330A000A00B99
:100210000729000000000130AE070318AF0A0329C8
:100220008B16AF1B1A29AF08031D1D292E086A3C27
:10023000031C1D29AF016B30AE00AF1B2929AF088D
:10024000031D26292E08C53C03182929AF01C530F6
:10025000AE006430AE020030031C0130AF02AF1BB1
:100260003829AF08031D58292E082E3C031C582995
:100270000330B00034302E02A0002F08A30000305D
:10028000031C0130A3022008003CB400B501230880
:10029000031C230FB5023508B7003408B600B901B6
:1002A0000530B80077202208AF002108AE007D2974
:1002B000AF1B7929AF08031D61292E08393C0318AB
:1002C00079293030B00034302E02B4002F08B50048
:1002D0000030031C0130B5023508B7003408B60001
:1002E000B9010530B80077202208AF002108AE0020
:1002F0007D298501AF01AE0105152E08B200FE284B
:02030000630098
:02400E00C43CB0
:00000001FF
